:0200000480007A
:100000006F00C004732F2034930F8000630AFF0336
:10001000930F90006306FF03930FB0006302FF038A
:10002000170F0080130F0FFE63040F0067000F000F
:10003000732F203463540F006F004000136E9E53E3
:10004000171F00002320CFFD6FF09FFF732540F1A5
:100050006310050073251030635805000F00F00F82
:10006000130E100073000000130E00009702000032
:10007000938282F973905230735020307350303035
:1000800073504030970200809382C2F7638C020065
:10009000739052109302B01A739022307323203061
:1000A000E39E62F873500030970200009382420191
:1000B00073901234732540F173002030130E20002A
:1000C000930000001301000063D620006318C031C4
:1000D0006316C001E3DE20FE6312C031130E300050
:1000E000930010001301100063D620006318C02F86
:1000F0006316C001E3DE20FE6312C02F130E400022
:100100009300F0FF1301F0FF63D620006318C02DA9
:100110006316C001E3DE20FE6312C02D130E5000F3
:10012000930010001301000063D620006318C02B59
:100130006316C001E3DE20FE6312C02B130E6000C5
:10014000930010001301F0FF63D620006318C0294C
:100150006316C001E3DE20FE6312C029130E700097
:100160009300F0FF1301E0FF63D620006318C0275F
:100170006316C001E3DE20FE6312C027130E800069
:10018000930000001301100063D420006314C00129
:100190006316C025E3DE20FE130E90009300F0FFEF
:1001A0001301100063D420006314C0016318C0233E
:1001B000E3DE20FE130EA0009300E0FF1301F0FF2A
:1001C00063D420006314C001631AC021E3DE20FE63
:1001D000130EB0009300E0FF1301100063D4200061
:1001E0006314C001631CC01FE3DE20FE130EC000B9
:1001F000130200009300F0FF1301000063D0201EE3
:100200001302120093022000E31652FE130ED000D8
:10021000130200009300F0FF130100001300000020
:1002200063DE201A1302120093022000E31452FE30
:10023000130EE000130200009300F0FF1301000012
:10024000130000001300000063DA201813021200EC
:1002500093022000E31252FE130EF000130200007E
:100260009300F0FF130000001301000063D8201674
:100270001302120093022000E31452FE130E000139
:10028000130200009300F0FF1300000013010000B0
:100290001300000063D42014130212009302200004
:1002A000E31252FE130E1001130200009300F0FF40
:1002B00013000000130000001301000063D020129F
:1002C0001302120093022000E31252FE130E2001CB
:1002D000130200009300F0FF1301000063D0201010
:1002E0001302120093022000E31652FE130E300197
:1002F000130200009300F0FF130100001300000040
:1003000063DE200C1302120093022000E31452FE5D
:10031000130E4001130200009300F0FF13010000D0
:10032000130000001300000063DA200A1302120019
:1003300093022000E31252FE130E5001130200003C
:100340009300F0FF130000001301000063D82008A1
:100350001302120093022000E31452FE130E6001F8
:10036000130200009300F0FF1300000013010000CF
:100370001300000063D42006130212009302200031
:10038000E31252FE130E7001130200009300F0FFFF
:1003900013000000130000001301000063D02004CC
:1003A0001302120093022000E31252FE9300100089
:1003B00063DA000093801000938010009380100097
:1003C000938010009380100093801000930E3000F3
:1003D000130E80016394D001631CC0010F00F00F65
:1003E00063000E00131E1E00136E1E00730000003B
:1003F0000F00F00F130E100073000000731000C008
:0404000000000000F8
:1010000000000000000000000000000000000000E0
:1010100000000000000000000000000000000000D0
:1010200000000000000000000000000000000000C0
:1010300000000000000000000000000000000000B0
:081040000000000000000000A8
:040000058000200057
:00000001FF
